:1000000016C025C024C023C0B0C021C020C01FC05E
:100010001EC01DC01CC01BC01AC019C018C00038AB
:10002000003701010101010101020408102011241F
:100030001FBECFE5D2E0DEBFCDBF20E0A0E6B0E03E
:1000400001C01D92A936B207E1F7D6D036C1D8CF8C
:1000500090E0FC01E85DFF4F24918E5D9F4FFC0115
:100060008491882381F090E0FC01E05EFF4FA49131
:10007000B0E0825E9F4FFC0184918FB7F894EC91C1
:10008000E22BEC938FBF0895282F30E0F901E85D53
:10009000FF4F9491F901EE5DFF4FE491EE23A1F043
:1000A000811113C08AB58F738ABDF0E0E25EFF4F05
:1000B000A491B0E08FB761110BC0F8942C91E92F97
:1000C000E095E223EC938FBF08958AB58F7CECCF47
:1000D000F894EC91E92BF6CF3FB7F8948091650046
:1000E00090916600A0916700B09168002FB508B6A6
:1000F00002FE05C02F3F19F00196A11DB11D3FBFA3
:10010000BA2FA92F982F8827BC01CD01620F711D2E
:10011000811D911D42E0660F771F881F991F4A9528
:10012000D1F70895CF92DF92EF92FF92CF93DF93B2
:100130006B017C01D1DFEB01CFDF6C1B7D0B683ED7
:100140007340D0F381E0C81AD108E108F108C85122
:10015000DC4FC114D104E104F10471F7DF91CF91B8
:10016000FF90EF90DF90CF90089578941F920F92B8
:100170000FB60F9211242F933F938F939F93AF93BA
:10018000BF938091610090916200A0916300B09153
:100190006400309160002CE7230F2D3728F02FEFFB
:1001A000230F0196A11DB11D209360008093610073
:1001B00090936200A0936300B09364008091650007
:1001C00090916600A0916700B09168000196A11D12
:1001D000B11D8093650090936600A0936700B09373
:1001E0006800BF91AF919F918F913F912F910F9098
:1001F0000FBE0F901F901895789480B7806880BFCD
:1002000080B7806480BF8CB580648CBD8FEF8DBD5E
:1002100080B7807F876080BF89B7846089BF83B7DC
:10022000887F83BF8AB58C7F81608ABD83B7877FD3
:1002300083BF83B7887F836083BF86B1876086B9B9
:10024000379A81E005DF80E003DF61E080E01CDFBA
:10025000CFE1D0E0219789F061E081E015DF64EF24
:1002600071E080E090E05EDF60E081E00DDF64EF50
:1002700071E080E090E056DFEDCF60E080E004DFE9
:10028000CAE1D0E0219761E081F081E0FDDE64E623
:1002900070E080E090E046DF60E081E0F5DE64E65B
:1002A00070E080E090E03EDFEDCF80E0EDDE68EED4
:0E02B00073E080E090E036DFFACFF894FFCFE5
:00000001FF
